:047C00000C942A3E78
:147C540001E005BF02E005BFCFE5D8E0CDBFDEBFC051D0401B
:147C68000AEA08830024E0E6F0E010E0E43EF10711F0019231
:147C7C00FBCF0083E4E5FCE7A0E6B0E01CE7E435F10721F0C0
:147C9000C89531960D92F9CF64D1FFCF20D0F801209357005F
:147CA400E89508951AD0F901080131E030935700E895089580
:147CB800F80120FD20935700059114910895002E19E01093F6
:147CCC005700E895089505D0B1E1B0935700E8950895B091D7
:147CE0005700B0FDFCCF089501E217D119C01AD08091600025
:147CF400909161008F3FEFEF9E0709F410C02AD0002351F07E
:147D08004DD07FD0002319F001E203D105C000E400D102C0DC
:147D1C0000E4FDD0E6CF08950E94EC3F5F9BFECF6CB15F9BA5
:147D3000FECF4CB1362E242E309261002092600027E030E073
:147D440081010E94F83F10936300009362000E94CC3F08958B
:147D58000E94D53F222700274427552710C05F9BFECF84E609
:147D6C0090E0FA01E80FF91F2CB02082FA01E80FF91F208061
:147D8000220D4F5F5F4F4038E0E05E0760F35F9BFECF0CB1F0
:147D9400201711F401E001C000270E94D83F08950E94EC3FB3
:147DA8006627772717C084E690E0FB013196E80FF91F208079
:147DBC003324322C2224FB01E80FF91F40815527420D531DB1
:147DD0009B018A010E94543E6E5F7F4F6038E0E07E0728F3B1
:147DE40023E000916200109163000E944E3E25E0009162006B
:147DF800109163000E944E3E0E94693E0E94CC3F08950E9410
:147E0C00F03FAA24BB2423C0222700916200109163000A0D4C
:147E20001B1D0E945C3EB80184E690E0F5013196E80FF91F7B
:147E340020803324322C2224F501E80FF91F40815527420D0E
:147E4800531D0417150711F0002709C0C50102965C01C5010D
:147E5C008038E0E09E07C0F201E00E94CF3F08950E94F43F40
:147E700009E253D001E251D029C044275F9BFECFACB04A0D1E
:147E84005F9BFECF6CB1460FDA2CC62EC6018F3FEFEF9E079F
:147E980009F419C05F9BFECFACB04A0D5F9BFECF6CB1641727
:147EAC0069F42A2D860110D0860116D00A1519F401E22DD02E
:147EC00005C000E42AD002C000E427D0D6CF0E94D23F089579
:147ED400E199FECF1FBB0EBB2DBBE29AE19A0895E199FECFED
:147EE8001FBB0EBBE09A0DB308950E94D53F05E210D05F9B95
:147EFC00FECF4CB15F9BFECF2CB02094421521F4042F00951D
:147F10000E94633E0E94D83F08955D9BFECF0CB90895002776
:147F240011270F5F1F4F0030EDE71E07D4F308950E94D53FF2
:147F380005E4EFDF0EE6EDDF04E6EBDF03E5E9DF02E3E7DFAF
:147F4C004CB10E94D83F089581E085BF222425BE0C94000060
:147F60000895F89481E082BB22242AB82BB886E880BD20BCB4
:147F740088E18AB98FE289B94CB10EE3CCDFCFDF8CB18C3357
:147F880029F4D4DFADDE6EDFB0DFE0DFDFDF0895E2E00C9432
:147F9C00D93FE4E00C94D93FE8E00C94D93F5A934A93089556
:147FB000E1E049915991E0FD089569917991E1FD0895A99006
:147FC400B990E2FD0895C990D990E3FD0895E990F990089506
:147FD8007A936A930C94D53FBA92AA920C94EC3FDA92CA92BC
:127FEC000C94F03F222321F0000F111F2A95FACF0895FA
:00000001FF
